:0A15D70000010202030304040505ED
:1006A700E4F513F512F511F510C203C200C202C238
:1006B700011209E87E0F7F008E408F41754A0F7542
:1006C7004B12753E0F753F1C75460F754743754CAA
:1006D7000F754D5CEE54E070030207EB751400755F
:1006E70015808E168F17C374989FFF740F9ECF24A3
:1006F70002CF3400FEE48F0F8E0EF50DF50CF50BCF
:10070700F50AF509F508AF0FAE0EAD0DAC0CAB0B46
:10071700AA0AA909A808C312099E5026E515250BA0
:10072700F582E514350AF58374CDF0E50B2401F560
:100737000BE4350AF50AE43509F509E43508F50847
:1007470080C4E4F50BF50AF509F508AF0FAE0EAD59
:100757000DAC0CAB0BAA0AA909A808C312099E5035
:1007670031AE0AAF0BE5172FF582E5163EF583E0AC
:10077700FDE5152FF582E5143EF583EDF0EF240135
:10078700F50BE43EF50AE43509F509E43508F50803
:1007970080B985144085154174002480FF740F3497
:1007A700FFFEC3E54B9FF54BE54A9EF54AC3E5437C
:1007B7009FF543E5429EF542C3E5459FF545E54470
:1007C7009EF544C3E53F9FF53FE53E9EF53EC3E5F5
:1007D700479FF547E5469EF546C3E54D9FF54DE531
:1007E7004C9EF54CD2E843D82090E668E04409F0E7
:1007F70090E65CE0443DF0D2AFD288D28AC2A8C26C
:10080700AA90E680E020E105D20812135B90E6800B
:10081700E054F7F0538EF8C203300105120483C287
:1008270001300329120EFE5024C20312142F200098
:100837001690E682E030E704E020E1EF90E682E000
:1008470030E604E020E0E412138A1215E912109C46
:0208570080C758
:1004830090E6B9E070030205341470030205B12449
:10049300FE700302063424FB700302052E1470035E
:1004A3000205281460731460762405600302069322
:1004B3001215EB400302069F90E6BBE024FE602288
:1004C30014603324FD601114602224067048E54053
:1004D30090E6B3F0E5418037E54A90E6B3F0E54BAB
:1004E300802DE54290E6B3F0E5438023E54490E6B2
:1004F300B3F0E545801990E6BAE0FF1213B6AA06F9
:10050300A9077B01EA494B600DEE90E6B3F0EF904B
:10051300E6B4F002069F0206981215C502069F1262
:100523000CF702069F12159E02069F1215B30206D0
:100533009F1215ED400302069F90E6B8E0247F600A
:100543001514601924027063A200E43325E0FFA2AE
:1005530002E4334F8041E490E740F0803F90E6BCF3
:10056300E0547EFF7E00E0D394807C0040047D0154
:1005730080027D00EC4EFEED4F24D7F58274153ECC
:10058300F583E493FF3395E0FEEF24A1FFEE34E619
:100593008F82F583E0540190E740F0E4A3F090E606
:1005A3008AF090E68B7402F002069F0206981215F9
:1005B300EF400302069F90E6B8E024FE6016240293
:1005C300600302069F90E6BAE0B40105C20002068A
:1005D3009F02069890E6BAE0705590E6BCE0547E20
:1005E300FF7E00E0D394807C0040047D0180027D87
:1005F30000EC4EFEED4F24D7F58274153EF583E4EF
:1006030093FF3395E0FEEF24A1FFEE34E68F82F5EE
:1006130083E054FEF090E6BCE05480131313541FA0
:10062300FFE0540F2F90E683F0E04420F0806D80CC
:10063300641215F1506690E6B8E024FE60192402B6
:10064300705A90E6BAE0B40104D200804F90E6BA43
:10065300E064026047803E90E6BCE0547EFF7E008B
:10066300E0D394807C0040047D0180027D00EC4E49
:10067300FEED4F24D7F58274153EF583E493FF33E3
:1006830095E0FEEF24A1FFEE34E68F82F583800828
:10069300120080500790E6A0E04401F090E6A0E04D
:0306A3004480F0A0
:0106A6002231
:03000300021112D5
:10111200C0E0C083C082C0D075D000C004C005C08A
:1011220006C00790E6017443F0E535703790F00091
:1011320074AAF0A37411F0A374CCF0A374EEF0902F
:10114200E690E4F090E6917405F0300419AF2AAE0F
:1011520029AD28AC278F3D8E3C8D3B8C3A75390FDB
:10116200D20780021535A283B39283D007D006D06E
:0C11720005D004D0D0D082D083D0E03271
:03000B00020E647E
:100E6400C0E0C0F0C083C082C0D075D000C000C054
:100E740001C002C003C004C005C006C00785238C9E
:100E840085248AE5396016D2831539E539704C908A
:100E9400E600E054FDF0000000C283803E30073BD2
:100EA400AF3DAE3CAD3BAC3AEF24FFF53DEE34FF35
:100EB400F53CED34FFF53BEC34FFF53AE4FFFEFD81
:100EC400FCAB3DAA3CA93BA83AC312099E700CC2D4
:100ED4000790E600E04402F0000000D007D006D0FE
:100EE40005D004D003D002D001D000D0D0D082D01D
:060EF40083D0F0D0E032D3
:03003300020EFAC0
:040EFA0053D8EF32A8
:101454000123D101244A042700000000C107C1046C
:10146400012500043000000000042B0000000001EE
:021474002FBA8D
:10155C0085238C85248AE58954F04401F589438ED2
:06156C0008D28CD2A92276
:100F9A00F07F647E00121017902001E090E679F04D
:100FAA007F647E00121017902002E090E679F07FAD
:100FBA00647E00121017902003E090E679F07F64B7
:100FCA007E00121017902004E090E679F07F647E8C
:100FDA0000121017902005E090E679F07F647E00F9
:100FEA00121017902006E090E679F07F647E0012D6
:100FFA001017902007E090E679F07F647E001210C7
:0D100A0017902008E090E679F07F647E00EA
:0C101700EF4E6007EF1F70F81E80F522FE
:1014990090E6187408F000000090E619F0000000CA
:0F14A90090E61AF000000090E61BF00000002211
:1014B80090E6187409F000000090E619F0000000AA
:0F14C80090E61AF000000090E61BF000000022F2
:1009E80090E6007412F090E60B7403F0000000909B
:1009F800E6047480F00000007402F0000000740443
:100A0800F00000007406F00000007408F000000018
:100A1800E4F000000000000090E61274E8F0000026
:100A280000E490E613F000000090E614F0000000E7
:100A380090E615F000000090E6187408F000000039
:100A480090E619F000000090E61AF000000090E629
:100A58001BF000000090E6097404F000000090E626
:100A680070E04401F000000090E6727408F00000A5
:100A78000090E6207402F0000000E490E621F00007
:100A8800000090E602F000000090E603F090E60116
:100A98007443F043AF0100000090E61074A0F0002A
:100AA800000090E611F000000090E65EE04408F0D7
:100AB800000000E490E68DF090E65EE04404F0006B
:100AC8000000E490E68FF0D20043B20843B202750A
:100AD800B5F01215E190E67AE054FEF0E4F5B0C204
:100AE800817F64FE121017D28112155C751D207566
:100AF8001E337B027D107FA012140A902033E0F58C
:100B080038A3E0F526E5386401600BE53864026037
:100B180005E538B40505752FBAC206E538640360E3
:100B280005E538B40405752FB8C206E538640660D3
:100B380005E538B41605752F20D206E53864076038
:100B480005E538B40805752F30D206E538B409052F
:0B0B5800752FBAD206E4F535D28322D7
:10109C00E5256402706FC2832080FD7F057E0012FF
:1010AC0011DC90E600E054FDF085332E85322D8561
:1010BC00312C85302BE47F64FEFDFCAB2EAA2DA9D0
:1010CC002CA82BD312099E40217F647E001211DCC8
:1010DC00E52E249CF52EE52D34FFF52DE52C34FF63
:1010EC00F52CE52B34FFF52B80CBAE2DAF2E12114A
:1010FC00DC90E6017440F090E600E04402F0D2A8E7
:06110C00C283E4F5252278
:020EFE00D322FD
:0215E900D3220B
:0215EB00D32209
:10159E0090E680E030E704D2058002C20590E6BAFC
:0515AE00E0F534D3223A
:1015B30090E740E534F0E490E68AF090E68B04F09F
:0215C300D32231
:080CF70090E6BAE0F522D322D9
:1015C50090E740E522F0E490E68AF090E68B04F09F
:0215D500D3221F
:0215ED00D32207
:0215EF00D32205
:0215F100D32203
:1000800090E6B9E01209C200BBB300DFB70125B8A2
:10009000017FB9019DBB022CBD026CBF027BC00277
:1000A000A8C10303C20346C8036DC903BBCA03E862
:1000B000CB043ECD046DCF0000047FC2A890E601C2
:1000C0007440F000000090E6047480F000000074BA
:1000D00002F0000000E4F0000000D2A802045D90ED
:1000E000E6BDE0FE90E6BCE07C002400F519EC3EA5
:1000F000F518200617AD1990E6BEE0FB7EE7751DEA
:10010000E7751E40AF2F12140A0203D790E6BEE037
:10011000FB7EE7751EE7751F40AD19AC18AF2F12B7
:1001200013E20203D7E490E68AF090E68BF090E6C3
:10013000A0E020E1F9E4FFFE74402FF582E434E70B
:10014000F583E0FD74002FF582E43420F583EDF0B3
:100150000FBF00010EEF64134E70DD902000E070C1
:100160000312132C902000E0B4010312117E9020A2
:1001700000E064026003020481121477020481E447
:1001800090E68AF090E68BF090E6A0E020E1F9E5B9
:100190002FC313FF7AE77B407D03020439E490E626
:1001A0008AF090E68BF090E6A0E020E1F978137CED
:1001B000207D017B0120062D7AE679BC7E007F013F
:1001C00012092990E6BEE0FF7E0078147C207D01B4
:1001D0007B017AE77940120929E52FC313FF90E6E6
:1001E000BEE004803F7AE679BD7E007F01120929D6
:1001F00078147C207D017B017AE679BC7E007F014A
:1002000012092990E6BEE0FF7E0078157C207D0172
:100210007B017AE77940120929E52FC313FF90E6A5
:10022000BEE02402FD7A207B13020439E490E68AC2
:10023000F090E68BF090E6A0E020E1F990E740E056
:10024000FCA3E0FDA3E0FEA3E0F52A8E298D288C17
:1002500027E4FFFEFDFCAB2AAA29A928A827C31280
:10026000099E7004C204807ED204807AE4F539C20B
:100270000790E600E04402F000000090E6BAE030AB
:10028000E00E90E6BCE05490FFE5B0546F4FF5B03F
:1002900090E6BAE030E10E90E6BCE05460FFE5B0D5
:1002A000549F4FF5B0020474E490E68AF090E68B18
:1002B000F090E6A0E020E1F990E740E0FCA3E0FD4B
:1002C000A3E0FEA3E0F52A8E298D288C27E4FFFE0B
:1002D000FDFCAB2AAA29A928A827C312099E7004ED
:1002E000C2048002D204E4F539C20775350190E6F4
:1002F00000E04402F0000000E490E68AF000000014
:1003000002047990E74074F4F0A37417F0E4A3F0CA
:10031000A3F0A3F0A20633A3F0A3E526F0A3E52FF4
:10032000F0A3E538F0300505E4A3F0800690E74936
:1003300074FFF0000000E490E68AF000000090E610
:100340008B740A020467E490E68AF090E68BF090E2
:10035000E6A0E020E1F990E740E014600C14600BA7
:100360002402600302048180258032803FE490E60D
:100370008AF090E68BF090E6A0E020E1F990E7406B
:10038000E0146019146025240260030204817523BF
:10039000F475245390E6007402F00204817523E89A
:1003A0007524A590E600740AF00204817523D175C6
:1003B000244A90E6007412F002048190E6BCE075D5
:1003C0001800F519FD90E6BEE0FB7EE7751DE775A8
:1003D0001E407FA012140AE490E68AF0000000900C
:1003E000E6BEE090E68B807FE490E68AF090E68BB4
:1003F000F090E6A0E020E1F990E6BCE0D39407504D
:100400000302048178137C207D017B017AE679BCAC
:100410007E007F0112092990E6BEE0FF7E0078147D
:100420007C207D017B017AE7794012092990E6BEA4
:10043000E004FD7A207B137F501215108043E49076
:10044000E68AF090E68BF090E6A0E020E1F990E7F4
:1004500040E0700512149980031214B8E490E68A03
:10046000F000000090E68BF00000008014C28112C2
:100470001013D281E490E68AF090E68BF08002D3EC
:0204800022C395
:010482002257
:10152C00C0E0C083C082D2015391EF90E65D74019C
:08153C00F0D082D083D0E03230
:10157200C0E0C083C0825391EF90E65D7404F0D066
:0615820082D083D0E032AC
:10158800C0E0C083C0825391EF90E65D7402F0D052
:0615980082D083D0E03296
:10122200C0E0C083C08290E680E030E70E853E4297
:10123200853F43854644854745800C854642854720
:1012420043853E44853F455391EF90E65D7410F02F
:07125200D082D083D0E0320E
:10154400C0E0C083C082D2035391EF90E65D74087B
:08155400F0D082D083D0E03218
:10125900C0E0C083C08290E680E030E70E853E4260
:10126900853F43854644854745800C8546428547E9
:1012790043853E44853F455391EF90E65D7420F0E8
:07128900D082D083D0E032D7
:010CFF0032C2
:0115F30032C5
:0115F40032C4
:0115F50032C3
:10102300C0E0C083C082C0D075D000C000C004C07F
:1010330005C006C007C2AFE4FFFEFDE52BFC781830
:101043001209AF90E7C4EFF0E4FFFEE52CFDE4FCEA
:1010530078101209AFA3EFF0E4FFE52DFEE4FDFCE9
:1010630078081209AFA3EFF0E52EFFA3EFF000001D
:101073000090E68F7408F00000005391EF90E65F54
:10108300E04404F0D2AFD007D006D005D004D0009E
:09109300D0D0D082D083D0E0322D
:100DB800C0E0C083C082C0D075D000C004C005C0E8
:030DC80006C0075B
:100DCB00C2AF90E6A1E020E1F990E780E024EF606C
:100DDB002214604F2413605024EF705890E781E089
:100DEB00FCA3E0FDA3E0FEA3E0F5338E328D318C46
:100DFB00308041752501C2A8D28390E600E0440201
:100E0B00F000000090E6017440F000000090E60452
:100E1B007480F00000007402F0000000E4F00000A9
:100E2B00008011752502800C752E64752D00752CB4
:100E3B0000752B0000000090E68DE4F05391EF90CD
:080E4B00E65FE04408F0D2AFBD
:100E5300D007D006D005D004D0D0D082D083D0E044
:010E6300325C
:0115F60032C2
:0115F70032C1
:0115F80032C0
:0115F90032BF
:0115FA0032BE
:0115FB0032BD
:0115FC0032BC
:0115FD0032BB
:0115FE0032BA
:0115FF0032B9
:0116000032B7
:0116010032B6
:0116020032B5
:0116030032B4
:0116040032B3
:0116050032B2
:0116060032B1
:0116070032B0
:0116080032AF
:0116090032AE
:01160A0032AD
:01160B0032AC
:01160C0032AB
:01160D0032AA
:01160E0032A9
:01160F0032A8
:0116100032A7
:0116110032A6
:0116120032A5
:0116130032A4
:10132C0090E678E04480F090E679E52F1210129068
:10133C00200112100E90200212100E902003121099
:0F134C000E90E678E04440F07F647E00021017B8
:10117E0090E678E04480F090E679E52F1210127434
:10118E0001120F9A90200912100E90200A12100EC2
:10119E0090200B12100E90200C12100E90200D129B
:1011AE00100E90200E12100E90200F12100E902086
:1011BE001012100E90201112100E90201212100EFE
:0E11CE0090E678E04440F07F647E0002101747
:1014770090E678E04480F090E679E52F1210127438
:101487002B120F9A90E678E04440F07F647E0002CA
:0214970010172C
:04140A008F1A8B1C8E
:10140E00902035EDF0E51AC313FF7A207B357D0170
:10141E00121510E51AC313FFAB1EAA1DAD1C021444
:01142E00F4C9
:0413E2008F1A8B1DB6
:1013E600EC902035F0EDA3F0E51AC313FF7A207BCD
:1013F600357D02121510E51AC313FFAB1FAA1EADE9
:041406001D0214F4BB
:1014D700A907EC902013F0EDA3F0EAA3F0EBA3F03B
:0D14E700E9C313FF7A207B137D040215106A
:100F00001201000200000040181621090000010231
:100F100000010A060002000000400100090227004B
:100F200001010080FA0904000003FF00000007052A
:100F3000820200020007058102400000070501024D
:100F40004000000902190001010080FA09040000B4
:100F500001FF0000000705820240000004030904AD
:100F600014035100480059002D0043004300440081
:100F700020002000240351004800590035002D00B6
:100F8000490049002000200020002000200020000F
:0A0F900020002000200020000000D7
:10138A0090E682E030E004E020E60B90E682E0306E
:10139A00E119E030E71590E680E04401F07F147E21
:0C13AA00001211DC90E680E054FEF022FE
:10142F0090E682E044C0F090E681F043870100002F
:04143F000000002287
:10135B0030080990E680E0440AF0800790E680E0D0
:10136B004408F07FDC7E051211DC90E65D74FFF023
:0F137B0090E65FF05391EF90E680E054F7F02298
:1011DC008E188F1990E600E054187012E51924014E
:1011EC00FFE43518C313F518EF13F519801590E6C5
:1011FC0000E05418FFBF100BE51925E0F519E518B0
:10120C0033F518E5191519AE18700215184E60054E
:06121C0012144380EE22D3
:0815E100E4F553D2E9D2AF2278
:1012900090E678E020E6F9C2E990E678E04480F054
:1012A000EF25E090E679F090E678E030E0F990E61E
:1012B00078E04440F090E678E020E6F990E678E0C7
:0612C00030E1D6D2E92264
:1012FA00A90790E678E020E6F9E553702390E678AE
:10130A00E04480F0E925E090E679F08D4EAF03A93C
:10131A0007754F018A508951E4F552755301D3225A
:02132A00C322DC
:1012C600A90790E678E020E6F9E553702590E678E0
:1012D600E04480F0E925E0440190E679F08D4EAFD8
:1012E60003A907754F018A508951E4F552755303D6
:0412F600D322C3221A
:03004B00020B6342
:100B6300C0E0C083C082C085C084C086758600C0D3
:100B7300D075D000C000C001C002C003C006C007CA
:100B830090E678E030E206755306020C4D90E67865
:100B9300E020E10CE55364026006755307020C4D37
:100BA300E55324FE605F14603624FE7003020C3E9E
:100BB30024FC7003020C4A24086003020C4DAB4F63
:100BC300AA50A951AF5205528F8275830012094F63
:100BD30090E679F0E552654E7070755305806B9021
:100BE300E679E0AB4FAA50A951AE528E82758300CD
:100BF30012097C755302E54E6401704E90E678E06D
:100C03004420F08045E54E24FEB5520790E678E097
:100C13004420F0E54E14B5520A90E678E04440F0E3
:100C230075530090E679E0AB4FAA50A951AE528EAE
:100C33008275830012097C0552800F90E678E044A8
:100C430040F075530080037553005391DFD007D0F4
:100C530006D003D002D001D000D0D0D086D084D02B
:080C630085D082D083D0E0327D
:0213B600A90785
:1013B800AE4CAF4D8F828E83A3E064037017AD01EE
:1013C80019ED7001228F828E83E07C002FFDEC3EA8
:0913D800FEAF0580DF7E007F00FE
:0113E10022E9
:1014F4001212C6E55324FA600E146006240770F332
:0C150400D322E4F553D322E4F553D322A4
:101510001212FAE55324FA600E146006240770F3E1
:0C152000D322E4F553D322E4F553D32288
:101443007400F58690FDA57C05A3E582458370F9BC
:011453002276
:03004300020D00AB
:03005300020D009B
:100D000002152C000215880002157200021544001D
:100D10000212220002125900020CFF000215F30019
:100D20000215F4000215F50002102300020DB800B0
:100D30000215F6000215F7000215F8000215F90079
:100D40000215FA000215F3000215FB000215FC0063
:100D50000215FD000215FE000215FF00021600003C
:100D6000021601000215F3000215F3000215F3004C
:100D70000216020002160300021604000216050005
:100D800002160600021607000216080002160900E5
:100D900002160A0002160B0002160C0002160D00C5
:100DA00002160E0002160F000216100002161100A5
:080DB0000216120002161300E6
:03000000020C6B84
:0C0C6B00787FE4F6D8FD758153020CB2CE
:10085900E709F608DFFA8046E709F208DFFA803E81
:1008690088828C83E709F0A3DFFA8032E309F6086E
:10087900DFFA8078E309F208DFFA807088828C83D6
:10088900E309F0A3DFFA806489828A83E0A3F6088A
:10089900DFFA805889828A83E0A3F208DFFA804C64
:1008A90080D280FA80C680D4806980F2803380103B
:1008B90080A680EA809A80A880DA80E280CA8033A4
:1008C90089828A83ECFAE493A3C8C582C8CCC5831C
:1008D900CCF0A3C8C582C8CCC583CCDFE9DEE780EC
:1008E9000D89828A83E493A3F608DFF9ECFAA9F06B
:1008F900EDFB2289828A83ECFAE0A3C8C582C8CCC1
:10090900C583CCF0A3C8C582C8CCC583CCDFEADED9
:10091900E880DB89828A83E493A3F208DFF980CC3B
:1009290088F0EF60010E4E60C388F0ED2402B40434
:100939000050B9F582EB2402B4040050AF232345DB
:0609490082239008A9734F
:10094F00BB010CE58229F582E5833AF583E022505D
:10095F0006E92582F8E622BBFE06E92582F8E222A7
:0D096F00E58229F582E5833AF583E49322C1
:10097C00F8BB010DE58229F582E5833AF583E8F0B1
:10098C00225006E92582C8F622BBFE05E92582C85D
:02099C00F22245
:10099E00EB9FF5F0EA9E42F0E99D42F0E89C45F0AF
:0109AE002226
:1009AF00E8600FECC313FCED13FDEE13FEEF13FF26
:0309BF00D8F1224A
:1009C200D083D082F8E4937012740193700DA3A3C4
:1009D20093F8740193F5828883E4737402936860D8
:0609E200EFA3A3A380DFD8
:100C77000206A7E493A3F8E493A34003F68001F2E6
:100C870008DFF48029E493A3F85407240CC8C3337E
:100C9700C4540F4420C8834004F456800146F6DF4D
:100CA700E4800B0102040810204080901454E47E75
:100CB700019360BCA3FF543F30E509541FFEE49342
:100CC700A360010ECF54C025E060A840B8E493A309
:100CD700FAE493A3F8E493A3C8C582C8CAC583CA34
:100CE700F0A3C8C582C8CAC583CADFE9DEE780BEEC
:011476000075
:00000001FF
